S01900006F70656E626C745F73746D3332663736372E73726563F5
S3150800000000000820510B00081D0B00081F0B0008F4
S31508000010210B0008230B0008250B00080000000030
S31508000020000000000000000000000000270B000888
S31508000030290B0008000000002B0B00082D0B0008F8
S31508000040A10B0008A10B0008A10B0008A10B0008D2
S31508000050A10B0008A10B0008A10B0008A10B0008C2
S31508000060A10B0008A10B0008A10B0008A10B0008B2
S31508000070A10B0008A10B0008A10B0008A10B0008A2
S31508000080A10B0008A10B0008A10B0008A10B000892
S31508000090A10B0008A10B0008A10B0008A10B000882
S315080000A0A10B0008A10B0008A10B0008A10B000872
S315080000B0A10B0008A10B0008A10B0008A10B000862
S315080000C0A10B0008A10B0008A10B0008A10B000852
S315080000D0A10B0008A10B0008A10B0008A10B000842
S315080000E0A10B0008A10B0008A10B0008A10B000832
S315080000F0A10B0008A10B0008A10B0008A10B000822
S31508000100A10B0008A10B0008A10B0008A10B000811
S31508000110A10B0008A10B0008A10B0008A10B000801
S31508000120A10B0008A10B0008A10B0008A10B0008F1
S31508000130A10B0008A10B0008A10B0008A10B0008E1
S31508000140A10B0008A10B0008A10B0008A10B0008D1
S31508000150A10B0008A10B0008A10B0008A10B0008C1
S31508000160A10B0008A10B0008A10B0008A10B0008B1
S31508000170A10B0008A10B0008A10B00080000000055
S31508000180A10B0008A10B0008A10B0008A10B000891
S31508000190A10B0008A10B0008A10B0008A10B000881
S315080001A0A10B0008A10B0008A10B0008A10B000871
S315080001B0A10B0008A10B0008A10B0008A10B000861
S315080001C0A10B0008A10B000800000000A10B000805
S315080001D0A10B0008A10B0008A10B0008A10B000841
S315080001E0A10B0008A10B0008A10B0008A10B000831
S30D080001F0A10B0008A10B000891
S315080001F810B5054C237833B9044B13B10448AFF34B
S3150800020800800123237010BD500000200000000064
S315080002183859000808B5034B1BB103490348AFF31F
S31508000228008008BD00000000540000203859000866
S3150800023853B94AB9002908BF00281CBF4FF0FF3137
S315080002484FF0FF3000F072B9ADF1080C6DE904CE35
S3150800025800F006F8DDF804E0DDE9022304B070478B
S315080002682DE9F047089E04468846002B4BD18A425A
S31508000278154667D9B2FA82F24AB1C2F1200701FADD
S3150800028802F320FA07F7954047EA030894404FEA2D
S31508000298154E230CB8FBFEF71FFA85FC0EFB1788CC
S315080002A843EA084307FB0CF1994209D9EB1807F109
S315080002B8FF3080F01B81994240F21881023F2B4497
S315080002C85B1AA4B2B3FBFEF00EFB103344EA0344F0
S315080002D800FB0CFCA44509D92C1900F1FF3380F062
S315080002E80781A44540F2048102382C4440EA0740B5
S315080002F8A4EB0C0400271EB1D4400023C6E900432A
S315080003083946BDE8F0878B4209D9002E00F0EB8004
S315080003180027C6E9000138463946BDE8F087B3FA2A
S3150800032883F7002F47D18B4202D3824200F2FA8024
S31508000338841A61EB030301209846002EE0D0C6E92B
S315080003480048DDE702B9FFDEB2FA82F2002A40F079
S315080003588F80491B4FEA154E1FFA85F80127B1FB0E
S31508000368FEFC230C0EFB1C1143EA014308FB0CF1A7
S31508000378994207D9EB180CF1FF3002D2994200F2DC
S31508000388CD808446591AA3B2B1FBFEF00EFB1014B1
S3150800039843EA044408FB00F8A04507D92C1900F1DC
S315080003A8FF3302D2A04500F2B6801846A4EB08042B
S315080003B840EA0C409FE7C7F1200CBB4022FA0CFE26
S315080003C84EEA030E01FA07F420FA0CF521FA0CF3A3
S315080003D84FEA1E482543B3FBF8F92C0C08FB1933DA
S315080003E81FFA8EFA44EA034309FB0AF49C4202FA06
S315080003F807F200FA07F10BD91EEB030309F1FF30E0
S3150800040880F087809C4240F28480A9F102097344EF
S315080004181B1BADB2B3FBF8F008FB103345EA0344DF
S3150800042800FB0AFAA24508D91EEB040400F1FF33BB
S315080004386BD2A24569D90238744440EA0940A0FB40
S315080004480289A4EB0A044C45C2464B4654D351D0FC
S31508000458002E69D0B1EB0A0564EB030404FA0CFC18
S31508000468FD40FC404CEA0505C6E90054002747E765
S31508000478C2F1200320FA03F7954001FA02F021FA9F
S3150800048803F34FEA154E3843010CB3FBFEF71FFA80
S3150800049885F80EFB173341EA034107FB08F38B423D
S315080004A804FA02F407D9691807F1FF3C2FD28B42E0
S315080004B82DD9023F2944CB1A81B2B3FBFEF00EFBB5
S315080004C8103341EA034100FB08F38B4207D9691840
S315080004D800F1FF3C17D28B4215D902382944C91AAC
S315080004E840EA07473BE73746304609E70746E7E65F
S315080004F81846FBE64145ABD2B8EB020A69EB0E0291
S3150800050801381346A4E76046E9E7184695E76746BB
S31508000518D1E781467CE702382C4447E7ACF1020C60
S315080005282B442FE7384608E73746E9E6704700BF01
S3150800053830B583B0002502AC04F8015D00F0AEF8CA
S3150800054803F0C8F92146284600F0C0F89DF8073098
S31508000558012B01D003B030BD03F044FAFAE708B519
S3150800056803F0C6F908BD08B501F078FB08BD000018
S3150800057808B54FF40051064801F024FB012805D0B8
S3150800058800F042F8FFF7EFFF012008BD0020FCE75E
S315080005980008024008B5642000F006F808BD08B54A
S315080005A800F008F808BD0000014B1880704700BF26
S315080005B86C00002008B503F033F90F4B1B68984206
S315080005C810D30E4B1B7873B901220C4B1A70802175
S315080005D80B4801F0FEFA03F023F90A4B1B88184466
S315080005E8054B186008BD0022044B1A708021044880
S315080005F801F0EFFAEFE700BF700000206E00002058
S31508000608000402406C00002008B500228021024838
S3150800061801F0DFFA08BD00BF000402400B4B1B6857
S31508000628C3F3072050FA83F2C3F30740104400EBDC
S315080006381360002305E0054A1A441279104480B26B
S315080006480133372BF7D9404280B2704700000020A3
S3150800065808B5FFF7E3FF044B9B8F984201D00020AB
S3150800066808BD0120FCE700BF0000002008B5054BBF
S315080006781A68054B9A4201D0002008BDFFF7E8FF23
S31508000688FBE700BF00000020A2E742CE08B5FFF747
S31508000698C5FF014B988708BD0000002008B5FFF77D
S315080006A8E5FF68B9074B084A1A60002304E0054ABB
S315080006B81A44002111710133372BF8D9FFF7E6FFE1
S315080006C808BD00BF00000020A2E742CE38B505469F
S315080006D80C46FFF7CBFF034658B1372D8CBF0023CE
S315080006E80123002C08BF00231BB1034A15442A79A5
S315080006F82270184638BD00BF0000002030B58DB0FE
S3150800070800240794089409940A940B94284B1A6BA6
S3150800071842F004021A631A6B02F004020192019A63
S315080007281A6B42F080021A631A6B02F08002029270
S31508000738029A1A6B42F001021A631A6B02F0010256
S315080007480392039A1A6B42F002021A631A6B02F0B2
S3150800075802020492049A1A6B42F008021A631A6B88
S3150800076802F008020592059A1A6B42F040021A63CB
S315080007781B6B03F040030693069B0E4D2246802109
S31508000788284601F026FA4FF400530793089409946B
S3150800079807A9094801F088F88023079301230893D5
S315080007A809940A9407A9284601F07EF80DB030BDC9
S315080007B80038024000040240000802402DE9F041D2
S315080007C890B0002409940A940B940C940D940E94F2
S315080007D80F9406940794274B1A6C42F480221A64DD
S315080007E81A6C02F480220292029A1A6B42F00802E4
S315080007F81A631B6B03F008030193019B4FF480737C
S3150800080803934FF00208CDF81080032705970726AB
S315080008180896194D03A9284602F018F94FF40073EB
S315080008280393CDF81080059706940794089603A9AC
S31508000838284602F00BF94FF4E13309930A940B940E
S315080008480C940C230D930E940F940C4C09A920466E
S3150800085802F088FB636823F490436360A36823F077
S315080008682A03A360236843F00103236010B0BDE898
S31508000878F08100BF00380240000C024000480040E2
S3150800088830B5B9B0342200212BA805F049F8002460
S3150800089826942794289429942A949022214602A8D3
S315080008A805F03EF8204B1A6C42F080521A641B6C0D
S315080008B803F080530093009B1C4B1A6842F440428D
S315080008C81A601B6803F440430193019B01232B9389
S315080008D84FF4A0232C93022531954FF480033293C5
S315080008E8082333934FF4D8733493359536952BA844
S315080008F801F062FA01F074F90F23269327952894D4
S315080009084FF4A05329934FF480532A93072126A816
S3150800091801F0E0FC4FF480730293159402A801F0E5
S3150800092893FD39B030BD00BF003802400070004062
S3150800093808B500F06FF9FFF7A3FFFFF7DFFEFFF72B
S315080009483DFFFFF7F5FDFFF70AFEFCE782B00A4B05
S315080009581A6C42F080521A641A6C02F0805200929D
S31508000968009A5A6C42F480425A645B6C03F48043DA
S315080009780193019B02B0704700380240F0B58DB06C
S3150800098800230793089309930A930B9302683A4B33
S315080009989A4201D00DB0F0BDA3F590431A6B42F008
S315080009A800721A631A6B02F000720092009A1A6BA8
S315080009B842F080621A631A6B02F080620192019A09
S315080009C81A6B42F000621A631A6B02F0006202920E
S315080009D8029A1A6B42F004021A631A6B02F00402AE
S315080009E80392039A1A6B42F001021A631A6B02F011
S315080009F801020492049A1A6B42F002021A631A6BED
S31508000A0802F002020592059A1A6B42F040021A632E
S31508000A181B6B03F040030693069B322307930226B3
S31508000A28089603250A950B240B9407A9134800F082
S31508000A383BFF862307930896002709970A950B9480
S31508000A4807A90F4800F030FF4FF40053079308969C
S31508000A5809970A950B9407A90A4800F025FF4FF449
S31508000A6820530793089609970A950B9407A90648E9
S31508000A7800F01AFF8EE700BF008002400008024017
S31508000A8800000240000402400018024010B51E4C3F
S31508000A9800228021204601F09CF88021204600F09B
S31508000AA8F1FF4FF40051194800F0ECFF04F5006413
S31508000AB84FF48071204600F0E5FF4FF40071204698
S31508000AC800F0E0FF124B1A6C22F480221A641A6BA3
S31508000AD822F040021A631A6B22F008021A631A6B8C
S31508000AE822F004021A631A6B22F002021A631A6BBE
S31508000AF822F001021A631A6C22F080521A645A6CA0
S31508000B0822F480425A6410BD0004024000080240DC
S31508000B18003802407047FEE7FEE7FEE7FEE7704743
S31508000B287047704708B500F081F808BD054BD3F83B
S31508000B38882042F47002C3F888204FF000629A6051
S31508000B48704700BF00ED00E0DFF834D0002103E06D
S31508000B580C4B5B58435004310B480C4B42189A42CD
S31508000B68F6D30B4A02E0002342F8043B094B9A42A3
S31508000B78F9D3FFF7DBFF04F095FEFFF7D9FE7047B8
S31508000B8800000820545A00084000002050000020A1
S31508000B98500000204C3E0020FEE7000010B5094B27
S31508000BA84FF0FF321A6200241C625A625C621A61AC
S31508000BB81C615A615C619A619C61FFF767FF204670
S31508000BC810BD00BF0038024010B504460E4B187811
S31508000BD84FF47A73B3FBF0F30C4A1068B0FBF3F0E2
S31508000BE800F088F868B90F2C01D901200AE000221C
S31508000BF821464FF0FF3000F04BF8054B1C600020EB
S31508000C0800E0012010BD00BF44000020400000207D
S31508000C184800002008B5032000F028F80020FFF750
S31508000C28D3FFFFF793FE002008BD0000034A1168AA
S31508000C38034B1B780B441360704700BF74060020EB
S31508000C484400002038B5044602F0F2FD0546B4F122
S31508000C58FF3F02D0044B1B781C4402F0E9FD401BF9
S31508000C68A042FAD338BD00BF440000200649CB6825
S31508000C7823F4E0631B041B0C000200F4E060034342
S31508000C88024A1A43CA60704700ED00E00000FA05F8
S31508000C9830B4154BDB68C3F30223C3F10704042CED
S31508000CA828BF04241D1D062D14D9033B4FF0FF3514
S31508000CB805FA04F421EA0401994005FA03F322EA3D
S31508000CC803031943002807DB0901C9B2074B19545E
S31508000CD830BC70470023E9E700F00F000901C9B2E4
S31508000CE8034B1954F4E700BF00ED00E000E400E008
S31508000CF814ED00E00138B0F1807F0AD2064B58603F
S31508000D08064AF02182F823100020986007221A6004
S31508000D1870470120704700BF10E000E000ED00E0D2
S31508000D285079137943EA002307480B50D07893780B
S31508000D381B0443EA0063507843EA002312781343F6
S31508000D48024A8B50704700BF4080024044800240E8
S31508000D58016841F218028B5843F400538B507047C8
S31508000D68016841F218028B5843F002038B5070470A
S31508000D7870B59EB0044629B14FF40063C3604FF4BA
S31508000D8880438360E369002B68D14FF48063079337
S31508000D9821680B68374A1A40A368E068034307982E
S31508000DA8034343F4007313430B6023681D6801204B
S31508000DB8FFF748FF23681D60236840225A602368A6
S31508000DC85D680120FFF73EFF23685D6023680025FC
S31508000DD89D602368DD602268936923F0BE031B04BF
S31508000DE81B0C43F08003936123689E690120FFF773
S31508000DF829FF23689E612368DD612368DD69012070
S31508000E08FFF720FF2368DD61216841F218054B5971
S31508000E18194A1A40194B13434B5123685E59012046
S31508000E28FFF710FF23685E51236803F58053144AB9
S31508000E381A60236803F580531D680120FFF702FF2F
S31508000E48236803F580531D60A369012B09D06269DD
S31508000E5800212046FFF764FF1EB070BD00230793E4
S31508000E6896E7216841F21C028858064B03438B50C3
S31508000E78EDE700BF0F8120FF233FDEF804002002BC
S31508000E888020C1024000010010B582B00446002344
S31508000E9801930268136843F00803136003681B6824
S31508000EA801930120FFF7CEFE2368019A1A6002B063
S31508000EB810BD10B582B00446002301930268136872
S31508000EC843F00403136003681B6801930120FFF7C6
S31508000ED8B9FE2368019A1A6002B010BD30B583B00E
S31508000EE8054600230193026841F21804135943F48E
S31508000EF88013135103681B5901930120FFF7A2FEBB
S31508000F082B68019A1A5103B030BDF0B490F84540E1
S31508000F18012C31D0012480F84540022480F8444049
S31508000F28C162002401E0F96001349C4217D26501C8
S31508000F384F194FF480164E5140F2F45606FB042614
S31508000F48BE60C6691EB94E5946F440064E515D1E26
S31508000F58A542E8D9651C01EB4515FD60E4E702687A
S31508000F6841F21003D150012380F84430002380F859
S31508000F7845301846F0BC70470220FBE7F0B490F8F5
S31508000F884540012C2ED0012480F84540022480F8DB
S31508000F9844408162002401E0E96001349C4214D28D
S31508000FA866018D194FF000478F5144F2F4566E606A
S31508000FB840F2F45606FB0426AE605E1EA642EBD93E
S31508000FC8661C01EB4616EE60E7E7026841F20C0379
S31508000FD8D150012380F84430002380F8453018465C
S31508000FE8F0BC70470220FBE790F84530012B00F06B
S31508000FF88580012380F84530022380F84430B1B152
S31508001008C36A1A68002A1ADB30B440F2F4529142CD
S315080010181DD93B4AA2FB0142920A40F2F45404FB4A
S31508001028121404B10132012A11D0002347E0012322
S3150800103880F84430002280F8452018467047122365
S3150800104880F84430002380F84530012070471A6834
S3150800105842F040521A60C36AC1F30C015960C26A69
S31508001068136843F000431360C36ADB68C362036806
S3150800107841F214029A5812F0040F08D041F21402E9
S3150800108804219950026841F204030021D150012332
S3150800109880F84430002380F84530184630BC70473D
S315080010A8C56A2C6844F080542C6011E0C56A2C681F
S315080010B844F000442C60C46AE468C46201339A4266
S315080010C8D5D9C56A2C6824F040542C60002BE7D083
S315080010D8C46A40F2F4556560541E9C42E6D1C56A56
S315080010E82C6844F000542C60064C04FB021404F2E5
S315080010F8F454C56AC4F30C046C60D7E70220704739
S315080011080BB002AC0CFAFFFF90F84530012B40D023
S31508001118012380F84530022380F84430836A1A6828
S31508001128002A28DB1A6812F4807F19D0826B0132EC
S315080011388263012A12D043631A68C2F30D42043A3D
S31508001148C263026B92680264DB688362012380F8D3
S315080011584430002380F84530184670470363EAE7A9
S315080011681A6812F4007F0ED0036300224263012234
S315080011788263DB688362012380F84430002280F8A2
S31508001188452018467047826B01328263DB688362A2
S31508001198F1E702207047F8B590F84430DBB2822BA5
S315080011A833D016460546822380F844300268136908
S315080011B803F01C03048AE402A4B223438C0104F452
S315080011C8F8641C4344F00104146102F031FB074635
S315080011D814F0010F10D002F02BFBC01BB0F5803FAE
S315080011E802D22B681C69F3E7012385F844300023EB
S315080011F885F84530032007E02B685B699BB23360A6
S31508001208012385F844300020F8BD0220FCE790F851
S315080012184430DBB2422B32D070B50546422380F8FB
S3150800122844300068036903F01C032C8AE402A4B25C
S3150800123823438C0104F4F8641C4344F0030492B273
S3150800124842612B681C6102F0F3FA064614F0010F96
S3150800125810D002F0EDFA801BB0F5803F02D22B6859
S315080012681C69F3E7012385F84430002385F84530DF
S31508001278032003E0012385F84430002070BD0220CE
S315080012887047000070B582B000230193002800F06B
S315080012980C81044690F84430002B32D0844B5A6CA3
S315080012A842F480425A645B6C03F480430093009BC3
S315080012B8804B5A6822F400025A605A68216A0A431F
S315080012C85A60236803F580531A6842F001021A60C7
S315080012D802F0AEFA0546236803F58052126812F042
S315080012E8010F13D002F0A4FA401BB0F5FA7FF2D921
S315080012F8032584F84450002384F84530284602B06C
S3150800130870BD80F84530FFF739FBC7E71D6925F03A
S315080013181C0501F093F8684B0344684A934255D86C
S3150800132845F0080523681D614FF400420021204650
S31508001338FFF76DFF0546002860D1FF20FFF782FCFE
S315080013486368002B00F0918002F072FA064601AA3B
S3150800135801212046FFF71FFF02F06AFA801B41F2B7
S315080013688833984252D8019B13F0040FEFD04FF4F4
S31508001378805200212046FFF74AFF002852D102F082
S3150800138857FA064601AA01212046FFF704FF02F08C
S315080013984FFA801B41F2883398424BD8019B13F0C9
S315080013A8200FEFD001AA1F212046FFF7F4FE0028D8
S315080013B84CD1019B13F0100F50D04FF40062E26035
S315080013C813F0040F4DD00023A3605EE03C4B0344A2
S315080013D83C4A934202D845F00C05A3E73A4B034426
S315080013E83A4A93429ED93A4B03443A4A934202D818
S315080013F845F0040596E745F0100593E701212046D0
S31508001408FFF7B6FC012584F8445077E70121204602
S31508001418FFF7AEFC012384F84430002384F84530EE
S3150800142803256BE701212046FFF7A2FC012584F86E
S31508001438445063E701212046FFF79AFC012384F804
S315080014484430002384F84530032557E70121204610
S31508001458FFF78EFC012584F844504FE70022E26026
S31508001468AEE74FF48043A3600FE0E268C2F3CF0209
S31508001478A368C3F34F031A4300212046FFF7C7FEA4
S3150800148858B940F6FF70FFF7DDFB00212046FFF745
S315080014986FFC012384F8443030E701212046FFF722
S315080014A867FC012584F8445028E7012526E700BF8C
S315080014B8003802400038014000D3CEFEBFE1E40000
S315080014C840F1E9FD3F787D0100796CFCFF5962021D
S315080014D8001F0AFA7FF0FA0238B590F84530012B52
S315080014E81AD00446012580F84550022380F844306E
S315080014F8FFF7CAFC2046FFF7DCFC2046FFF7EEFCA0
S315080015082046FFF725FC2046FFF72AFC84F84450B6
S31508001518002084F8450038BD0220FCE710B40A49C3
S315080015280C6924F440740C610C6944F440740C6129
S315080015380C6944F001040C6102604360BFF34F8FE5
S315080015485DF8044B704700BF003C0240084B1A6917
S3150800155822F440721A611A6942F400721A611A6909
S3150800156842F001021A610160BFF34F8F704700BF4E
S31508001578003C0240084B1A6922F440721A611A693B
S3150800158842F480721A611A6942F001021A610180EE
S31508001598BFF34F8F704700BF003C0240074B1A69DC
S315080015A822F440721A611A691A611A6942F001022C
S315080015B81A610170BFF34F8F704700BF003C0240A5
S315080015C81A4BDB6813F0020F04D0194A936943F0E3
S315080015D820039361154BDB6813F0100F04D0144AE7
S315080015E8936943F010039361104BDB6813F0200FDF
S315080015F804D00F4A936943F0080393610B4BDB68E1
S3150800160813F0400F04D00A4A936943F00403936120
S31508001618064BDB6813F0800F04D0054A936943F03C
S3150800162802039361014BF222DA607047003C0240DC
S3150800163878060020094B1B69002B01DB0020704740
S31508001648064B074A5A6002F188325A601B69002B12
S3150800165801DB002070470120704700BF003C0240AC
S3150800166823016745034A136943F0004313610020C1
S31508001678704700BF003C024038B50446164B0022A6
S315080016889A6102F0D5F80546144BDB6813F4803FD7
S315080016980AD0B4F1FF3FF7D0CCB102F0C9F8401B25
S315080016A8A042F1D903200DE00C4BDB6813F0F20FCA
S315080016B809D10A4BDB6813F0010F0AD0074B012240
S315080016C8DA60002038BDFFF77BFF0120FAE7032020
S315080016D8F8E70020F6E700BF78060020003C02403D
S315080016E8F8B51E4C247D012C35D01F4616460D46E6
S315080016F804461A4B01221A754CF25030FFF7BCFF04
S31508001708014698B9032C07D8DFE804F002151A1F12
S31508001718F1B22846FFF742FF4CF25030FFF7ACFF0C
S3150800172801460F4A136923F0010313610B4B002284
S315080017381A750846F8BDB1B22846FFF71BFFEBE74E
S3150800174831462846FFF702FFE6E732463B46284673
S31508001758FFF7E4FEE0E70221EBE700BF7806002082
S31508001768003C0240114A136923F4407313610329A4
S3150800177810D0022914D00D4A136943F004031361E3
S315080017880A4A136943EA002040F480301061BFF31F
S315080017984F8F7047116948F204030B431361EFE74B
S315080017A8024A136943F400431361E9E7003C02401F
S315080017B810B449B1012926D0022902D04FF4407441
S315080017C803E04FF4007400E000240B2800D9043025
S315080017D80E4B196921F4407119611A6922431A6175
S315080017E81A6922F0F8021A611A6942EAC00040F03A
S315080017F8020018611A6942F480321A61BFF34F8FE2
S315080018085DF8044B70474FF48074DEE7003C0240ED
S31508001818224B1B7D012B3DD070B50E4604461F4B47
S3150800182801221A754CF25030FFF726FF024660BBB4
S315080018384FF0FF3333602368012B16D0A568E36899
S31508001848A1680B44AB4220D9217C2846FFF7B0FF94
S315080018584CF25030FFF710FF114A136923F0FA03C8
S315080018681361024680B90135E9E76168207CFFF70C
S3150800187879FF4CF25030FFF7FFFE0246084908691F
S31508001888084B03400B6100E03560044B00211975CD
S31508001898104670BD02221046704700BF7806002021
S315080018A8003C0240FB7FFFFF00230F2B00F2E1807C
S315080018B8F0B583B039E0092200E00022B2403A4385
S315080018C802346C4E46F824206B4A1468EA4302EA46
S315080018D804064F6817F4803F01D045EA0406664CAB
S315080018E82660646802EA04064F6817F4003F01D0C8
S315080018F845EA0406604C6660A46802EA04064F686E
S3150800190817F4801F01D045EA04065B4CA660E46814
S3150800191822404E6816F4001F01D045EA0402564CC8
S31508001928E26001330F2B00F2A28001229A400C686C
S3150800193804EA0205AA42F4D14C68661E112C18BF9F
S31508001948012E01D9122C12D186685F000324BC40E7
S3150800195826EA0406CC68BC4034438460466826EA0E
S3150800196802064C68C4F300129A4032434260C268C1
S315080019785F000326BE40F64332408C68BC401443D9
S31508001988C4604A68122A18BF022A13D1DC08083428
S3150800199850F824E003F007024FEA820C0F2202FAF5
S315080019A80CF22EEA020E0A6902FA0CF242EA0E0252
S315080019B840F82420026816404A6802F00302BA4032
S315080019C8324302604A6812F0805FAAD02B4A546CE8
S315080019D844F480445464526C02F480420192019A99
S315080019E89C08A61C234A52F8267003F003029600A0
S315080019F80F22B24027EA0207214A90423FF45DAF18
S31508001A0802F58062904222D002F58062904220D088
S31508001A1802F5806290421ED002F5806290421CD080
S31508001A2802F5806290421AD002F58062904218D078
S31508001A3802F58062904216D002F58062904214D070
S31508001A4802F5806290423FF436AF0A2236E7012251
S31508001A5834E7022232E7032230E704222EE705227A
S31508001A682CE706222AE7072228E7082226E703B0F2
S31508001A78F0BD704700380140003C0140003802407C
S31508001A880000024000230F2B00F29480F0B529E0ED
S31508001A98092700E0002707FA05F5B54271D0056859
S31508001AA85E000324B440E44325400560DD08083594
S31508001AB850F8256003F007074FEA870C0F2707FA3F
S31508001AC80CF726EA070640F82560C5682540C5606C
S31508001AD8456825EA02024260826814408460013338
S31508001AE80F2B66D801229A4002EA0104A242F6D1CF
S31508001AF84FEA930E0EF102062F4D55F8266003F0AD
S31508001B080305AD004FF00F0C0CFA05FC0CEA0606A7
S31508001B182A4FB842BED007F58067B84221D007F5E4
S31508001B288067B8421FD007F58067B8421DD007F509
S31508001B388067B8421BD007F58067B84219D007F501
S31508001B488067B84217D007F58067B84215D007F5F9
S31508001B588067B84213D007F58067B84298D00A2735
S31508001B6899E7012797E7022795E7032793E70427C5
S31508001B7891E705278FE706278DE707278BE70827C5
S31508001B8889E70F4D2E68E44326402E606E68264086
S31508001B986E60AE682640AE60EE683440EC60064E6D
S31508001BA80EF1020456F8245025EA0C0546F8245086
S31508001BB875E7F0BD704700BF0038014000000240D5
S31508001BC8003C01400369194201D1002070470120F1
S31508001BD8704712B90904816170478161704700002E
S31508001BE810B582B01B4B1A6C42F080521A641B6CF3
S31508001BF803F080530193019B174A136843F4803313
S31508001C08136001F015FE0446134B5B6813F4803F16
S31508001C1808D101F00DFE001BB0F57A7FF4D9032030
S31508001C2802B010BD0C4A136843F40033136001F080
S31508001C38FFFD0446084B5B6813F4003F07D101F023
S31508001C48F7FD001BB0F57A7FF4D90320E8E70020F2
S31508001C58E6E700BF003802400070004038B501F0DA
S31508001C68E7FD04464F4A136843F0010313604D4BDA
S31508001C781B6813F0020F07D101F0DAFD001B0228D2
S31508001C88F5D90323184638BD464D2B6843F080031B
S31508001C982B6001F0CDFD04460023AB60414B9B68E1
S31508001CA813F00C0F08D001F0C3FD001B41F288336E
S31508001CB89842F3D90323E5E701F0BAFD0446394A01
S31508001CC8136823F450231360364B1B6813F4003F3C
S31508001CD806D001F0ADFD001B6428F5D90323D1E72A
S31508001CE801F0A6FD04462F4A136823F08073136093
S31508001CF82C4B1B6813F0007F06D001F099FD001BDA
S31508001D080228F5D90323BDE701F092FD0446254AC2
S31508001D18136823F080631360224B1B6813F0006F67
S31508001D2806D001F085FD001B6428F5D90323A9E729
S31508001D3801F07EFD04461B4A136823F0805313609E
S31508001D48184B1B6813F0005F06D001F071FD001BE5
S31508001D586428F5D9032395E7124B134A5A60103AB3
S31508001D68C3F88420C3F88820DA6822F4FE42DA60C9
S31508001D78DA6842F47F02DA605A6F22F001025A677B
S31508001D885A6F42F080725A67084B094A1A60094B1B
S31508001D981868FEF719FF034600283FF473AF0123B6
S31508001DA870E700BF003802401030002440000020C9
S31508001DB80024F40048000020002800F0128270B5BC
S31508001DC882B00446036813F0010F29D0A24B9B681A
S31508001DD803F00C03042B1AD09F4B9B6803F00C03E3
S31508001DE8082B0FD06368B3F5803F40D0002B54D139
S31508001DF8994B1A6822F480321A601A6822F48022EB
S31508001E081A6039E0944B5B6813F4800FEAD0924B5A
S31508001E181B6813F4003F03D06368002B00F0E381C6
S31508001E28236813F0020F75D08B4B9B6813F00C0FC1
S31508001E385ED0894B9B6803F00C03082B53D0E368E4
S31508001E48002B00F08A80844A136843F00103136064
S31508001E5801F0EEFC0546804B1B6813F0020F73D1A0
S31508001E6801F0E6FC401B0228F5D90320BEE17A4AB0
S31508001E78136843F48033136063682BB301F0D8FC06
S31508001E880546754B1B6813F4003FC9D101F0D0FC11
S31508001E98401B6428F5D90320A8E1B3F5A02F09D07B
S31508001EA86D4B1A6822F480321A601A6822F4802266
S31508001EB81A60E1E7684B1A6842F480221A601A68C1
S31508001EC842F480321A60D7E701F0B2FC0546624B45
S31508001ED81B6813F4003FA3D001F0AAFC401B642832
S31508001EE8F5D9032082E15C4B5B6813F4800FA6D111
S31508001EF8594B1B6813F0020F04D0E368012B01D075
S31508001F08012073E1544A136823F0F803216943EA68
S31508001F18C1031360236813F0080F46D0636983B3B7
S31508001F284D4A536F43F00103536701F081FC054698
S31508001F38494B5B6F13F0020F37D101F079FC401B50
S31508001F480228F5D9032051E1434A136823F0F80318
S31508001F58216943EAC1031360DCE73F4A136823F0A3
S31508001F680103136001F064FC05463B4B1B6813F03C
S31508001F78020FCFD001F05CFC401B0228F5D90320DC
S31508001F8834E1354A536F23F00103536701F050FCD7
S31508001F980546314B5B6F13F0020F06D001F048FC7B
S31508001FA8401B0228F5D9032020E1236813F0040F03
S31508001FB87ED0294B1B6C13F0805F1ED1264B1A6CFA
S31508001FC842F080521A641B6C03F080530193019BFC
S31508001FD80125224B1B6813F4807F10D0A368012BB8
S31508001FE821D0002B3CD11C4B1A6F22F001021A672C
S31508001FF81A6F22F004021A671AE00025E9E7174A59
S31508002008136843F48073136001F012FC0646134BF9
S315080020181B6813F4807FE1D101F00AFC801B642851
S31508002028F5D90320E2E00C4A136F43F0010313675E
S31508002038A3685BB301F0FCFB0646074B1B6F13F05E
S31508002048020F34D101F0F4FB801B41F28833984221
S31508002058F3D90320CAE000BF0038024000700040E8
S31508002068052B09D0644B1A6F22F001021A671A6FFA
S3150800207822F004021A67DBE75F4B1A6F42F0040284
S315080020881A671A6F42F001021A67D1E701F0D0FB06
S315080020980646594B1B6F13F0020F08D001F0C8FB10
S315080020A8801B41F288339842F3D903209EE0FDB994
S315080020B8A369002B00F099804F4A926802F00C0237
S315080020C8082A59D0022B19D04B4A136823F0807373
S315080020D8136001F0ADFB0446474B1B6813F0007FFD
S315080020E848D001F0A5FB001B0228F5D903207DE09E
S315080020F8414A136C23F080531364D9E73E4A1368A0
S3150800210823F08073136001F093FB05463A4B1B686E
S3150800211813F0007F06D001F08BFB401B0228F5D987
S31508002128032063E0E369226A1343626A43EA821377
S31508002138A26A5208013A43EA0243E26A43EA026398
S31508002148226B43EA02732C4A5360136843F0807380
S31508002158136001F06DFB0446274B1B6813F0007FDC
S3150800216806D101F065FB001B0228F5D903203DE0DE
S3150800217800203BE0002039E01F4A5268012B37D07F
S3150800218802F48003E1698B4201D001202EE002F0B7
S315080021983F03216A8B4201D0012027E0616A47F68E
S315080021A8C0731340B3EB811F01D001201EE002F46F
S315080021B84031A36A5B08013BB1EB034F01D001200C
S315080021C814E002F07063E16AB3EB016F01D00120F5
S315080021D80CE002F0E042236BB2EB037F0AD0012041
S315080021E804E001207047012000E0002002B070BD1D
S315080021F80120FBE70020F9E700380240324B9B68CC
S3150800220803F00C03042B5CD0082B01D02F48704729
S315080022182DE9F04B2C4B5A6802F03F025B6813F421
S31508002228800F2BD0284B5B68C3F388131E460027FC
S315080022385C010025E41A65EB0705A90141EA9461E2
S31508002248A001001B61EB0501CB0043EA5073C400EB
S31508002258A01943EB07014B0243EAD0534402204630
S3150800226819460023FDF7E4FF174B5B68C3F30143E0
S3150800227801335B00B0FBF3F0BDE8F08B124B5B68EB
S31508002288C3F388131E4600275C010025E41A65EB8C
S315080022980705A90141EA9461A001001B61EB050144
S315080022A8CB0043EA5073C400A01943EB07018B021D
S315080022B843EA90538402204619460023FDF7B8FFDF
S315080022C8D2E70348704700BF003802400024F400EC
S315080022D800127A00002800F0A38070B50446524B15
S315080022E81B6803F00F038B420CD24F4A136823F07E
S315080022F80F030B431360136803F00F038B4201D0D7
S31508002308012070BD236813F0020F17D013F0040FCD
S3150800231804D0464A936843F4E0539360236813F05D
S31508002328080F04D0414A936843F4604393603F4AD0
S31508002338936823F0F003A068034393600D46236867
S3150800234813F0010F31D06368012B20D0022B25D05A
S31508002358364A126812F0020F64D034498A6822F0A5
S31508002368030213438B6001F063FA06462F4B9B68FA
S3150800237803F00C036268B3EB820F16D001F058FA23
S31508002388801B41F288339842F0D90320B9E7274AD7
S31508002398126812F4003FE0D10120B2E7234A126816
S315080023A812F0007FD9D10120ABE71F4B1B6803F059
S315080023B80F03AB420CD91C4A136823F00F032B43AF
S315080023C81360136803F00F03AB4201D0012098E7A6
S315080023D8236813F0040F06D0144A936823F4E053CD
S315080023E8E1680B439360236813F0080F07D00F4A78
S315080023F8936823F46043216943EAC1039360FFF7AE
S31508002408FDFE0A4B9B68C3F30313094AD35CD840FD
S31508002418084B1860084B1868FEF7D6FB002070E7CB
S315080024280120704701206CE7003C02400038024052
S31508002438505900084000002048000020014B186841
S31508002448704700BF40000020F0B583B00446036813
S3150800245813F0010F0CD0B54B9A6822F400029A6063
S315080024689A68416B0A439A60436BC3B1002600E039
S315080024780026236813F4002F15D0AC4AD2F88C30FE
S3150800248823F44013E16B0B43C2F88C30E36BB3F5C6
S31508002498801F06D0002B00F04581002504E00126A0
S315080024A8E7E70126F6E70025236813F4801F0FD00F
S315080024B89E4AD2F88C3023F44003216C0B43C2F8A9
S315080024C88C30236CB3F5800F00F02E8103B90125F3
S315080024D8236813F0807F00D0012613F0200F40F000
S315080024E82781236813F0100F0CD0904BD3F88C2053
S315080024F822F08072C3F88C20D3F88C20A16B0A438B
S31508002508C3F88C20236813F4804F08D0874AD2F87A
S31508002518903023F44033616E0B43C2F89030236839
S3150800252813F4004F08D0814AD2F8903023F4402398
S31508002538A16E0B43C2F89030236813F4803F08D085
S315080025487A4AD2F8903023F44013E16E0B43C2F866
S315080025589030236813F4003F08D0744AD2F89030B4
S3150800256823F44003216F0B43C2F89030236813F015
S31508002578400F08D06D4AD2F8903023F00303616CF7
S315080025880B43C2F89030236813F0800F08D0674AC7
S31508002598D2F8903023F00C03A16C0B43C2F89030A4
S315080025A8236813F4807F08D0604AD2F8903023F065
S315080025B83003E16C0B43C2F89030236813F4007FAC
S315080025C808D05A4AD2F8903023F0C003216D0B433D
S315080025D8C2F89030236813F4806F08D0534AD2F8AB
S315080025E8903023F44073616D0B43C2F8903023682A
S315080025F813F4006F08D04D4AD2F8903023F440639C
S31508002608A16D0B43C2F89030236813F4805F08D095
S31508002618464AD2F8903023F44053E16D0B43C2F88A
S315080026289030236813F4005F08D0404AD2F89030F7
S3150800263823F44043216E0B43C2F89030236813F401
S31508002648800F08D0394AD2F8903023F08063A16FFA
S315080026580B43C2F89030236813F4001F0DD0334A91
S31508002668D2F8903023F00063E16F0B43C2F890303C
S31508002678E36FB3F1006F00F0C180236813F0080F09
S3150800268800D0012513F4802F08D0284AD2F89030B4
S3150800269823F04073616F0B43C2F89030236813F434
S315080026A8000F09D0214AD2F8903023F08053D4F885
S315080026B880100B43C2F89030236813F0806F09D056
S315080026C81A4AD2F8903023F00053D4F884100B43F2
S315080026D8C2F89030236813F0006F09D0134AD2F86D
S315080026E88C3023F00073D4F888100B43C2F88C306A
S315080026F8236813F0805F09D00C4AD2F88C3023F08F
S315080027088063D4F88C100B43C2F88C30002E77D12E
S315080027182368B3F1007F73D0002D40F004810020B0
S3150800272803B0F0BD0125BFE60126CFE60038024012
S31508002738B74B1A6C42F080521A641B6C03F080532C
S315080027480193019BB34A136843F48073136001F03D
S315080027586FF80746AF4B1B6813F4807F06D101F064
S3150800276867F8C01B6428F5D90320D9E7A84B1B6F5F
S3150800277813F4407315D0226B02F440729A4210D0B3
S31508002788A34B1A6F22F44072196F41F48031196706
S31508002798196F21F4803119671A671B6F13F0010F37
S315080027A812D1236B03F44072B2F5407F1DD0984AC4
S315080027B8936823F4F813936095490B6F226BC2F359
S315080027C80B0213430B678CE601F032F80746904B69
S315080027D81B6F13F0020FE4D101F02AF8C01B41F26F
S315080027E888339842F3D903209AE78948826822F4FD
S315080027F8F812894919400A438260DDE701253CE752
S31508002808834A136823F08063136001F011F80646BB
S315080028187F4B1B6813F0006F06D001F009F8801B80
S315080028286428F5D903207BE7236813F0010F13D032
S31508002838636B8BB9764AD2F88430D2F8841060680C
S3150800284803F4403343EA801301F070610B43A1682F
S3150800285843EA0173C2F88430236813F4002F03D0BF
S31508002868E26BB2F5801F06D013F4801F1ED0236CC6
S31508002878B3F5800F1AD1664AD2F88430D2F8841094
S31508002888606803F4403343EA8013E06843EA006368
S3150800289801F0E0410B43C2F88430D2F88C3023F0BB
S315080028A81F03616A01390B43C2F88C30236813F099
S315080028B8807F11D0564AD2F88400D2F88410666808
S315080028C823691B0443EA861300F07060034301F08A
S315080028D8E0410B43C2F88430236813F0007F0DD01B
S315080028E8626823691B0443EA8213E26843EA0263BF
S315080028F8A26843EA0273464AC2F88430444A13680F
S3150800290843F08063136000F093FF0646404B1B684C
S3150800291813F0006F7FF400AF00F08AFF801B64286D
S31508002928F4D90320FCE63A4A136823F08053136067
S3150800293800F07EFF0546364B1B6813F0005F06D08D
S3150800294800F076FF401B6428F5D90320E8E62368DB
S3150800295813F4002F01D0E26B22B113F4801F1DD0A7
S31508002968236CDBB92A4AD2F88830D2F8881060690D
S3150800297803F4403343EA8013A06943EA006301F08D
S31508002988E0410B43C2F88830D2F88C3023F4F85368
S31508002998A16A013943EA0123C2F88C30236813F483
S315080029A8001F03D0E36FB3F1006F37D0236813F025
S315080029B8080F19D0164AD2F88810D2F888306069F4
S315080029C803F4403343EA801301F070610B43E1696D
S315080029D843EA0173C2F88830D2F88C3023F44033BE
S315080029E8E16A0B43C2F88C30094A136843F08053EE
S315080029F8136000F01DFF0446054B1B6813F0005FC3
S31508002A081FD100F015FF001B6428F5D9032087E6B7
S31508002A180038024000700040FFFCFF0F0A4AD2F84F
S31508002A288800D2F888106569236A1B0443EA851367
S31508002A3800F07060034301F0E0410B43C2F88830A8
S31508002A48B4E700206CE600BF00380240F0B40A6814
S31508002A5892FAA2F2B2FA82F22DE00E69C46893FAE3
S31508002A68A3F5B5FA85F56D00032707FA05F524EAEF
S31508002A78050493FAA3F5B5FA85F56D0006FA05F582
S31508002A882C43C4604C68022C40D04C68056893FAFD
S31508002A98A3F6B6FA86F67600032707FA06F625EAAF
S31508002AA8060593FAA3F3B3FA83F35B0004FA03F370
S31508002AB82B43036001320B6833FA02F45AD0012417
S31508002AC894402340F6D04C68013C012CC5D88E6842
S31508002AD8846893FAA3F5B5FA85F56D00032707FA0E
S31508002AE805F524EA050493FAA3F5B5FA85F56D0004
S31508002AF806FA05F52C4384600E68CD68446824EA0E
S31508002B08060405FB06F52C434460A6E793FAA3F4E6
S31508002B18B4FA84F4072C15D84E69046A93FAA3F50F
S31508002B28B5FA85F5AD000F2707FA05F524EA050471
S31508002B3893FAA3F5B5FA85F5AD0006FA05F52C431B
S31508002B480462A2E74D69466A1C0A94FAA4F7B7FA1A
S31508002B5887F7BF004FF00F0C0CFA07F726EA0706A7
S31508002B6894FAA4F4B4FA84F4A40005FA04F43443F1
S31508002B7844628AE70020F0BC70470000034B9B6854
S31508002B88C3F30313024AD35CD8407047003802409F
S31508002B9850590008034B9B68C3F38223024AD35C47
S31508002BA8D84070470038024060590008034B9B68B4
S31508002BB8C3F34233024AD35CD84070470038024010
S31508002BC8605900080D4B5B6803F480030BB90C4881
S31508002BD800E00C48094A536803F03F03B0FBF3F3D7
S31508002BE85068C0F3881000FB03F05368C3F3014329
S31508002BF801335B00B0FBF3F0704700BF00380240B2
S31508002C080024F40000127A0008B5074B9B6803F005
S31508002C180C03042B06D0082B01D0044808BDFFF77F
S31508002C28D1FFFBE70248F9E7003802400024F40020
S31508002C3800127A0008B5032808D00C282DD0B0F55C
S31508002C48406F51D0302877D0002008BD584BD3F8AC
S31508002C589030034043EA0040564B98420FD0B0F1F3
S31508002C68031F13D0013B984206D0FFF7CDFFFFF7A5
S31508002C7885FFFFF79BFFE8E7FFF7C6FFE5E74C4B3D
S31508002C881B6813F0020F7ED10020DEE7484B1B6F46
S31508002C9813F0020F79D10020D7E7454BD3F89030C7
S31508002CA8034043EA0040444B98420FD0B0F10C1F4A
S31508002CB813D0043B984206D0FFF7A6FFFFF75EFF3E
S31508002CC8FFF768FFC1E7FFF79FFFBEE7384B1B68AA
S31508002CD813F0020F5CD10020B7E7354B1B6F13F0D2
S31508002CE8020F57D10020B0E7314BD3F89030034094
S31508002CF843EA0040314B984210D0B0F10C2F14D05B
S31508002D08A3F58063984206D0FFF77EFFFFF736FFE4
S31508002D18FFF74CFF99E7FFF777FF96E7244B1B6801
S31508002D2813F0020F39D100208FE7214B1B6F13F0E0
S31508002D38020F34D1002088E71D4BD3F890300340A2
S31508002D4843EA00401E4B98420FD0B0F1301F13D00B
S31508002D58103B984206D0FFF757FFFFF70FFFFFF71C
S31508002D6819FF72E7FFF750FF6FE7114B1B6813F05F
S31508002D78020F17D1002068E70D4B1B6F13F0020FDF
S31508002D8812D1002061E70F485FE74FF400405CE77F
S31508002D980C485AE74FF4004057E70A4855E74FF4F6
S31508002DA8004052E7074850E74FF400404DE700BF98
S31508002DB8003802400200030008000C000008000C56
S31508002DC8200030000024F40008B5C0280AD0B0F561
S31508002DD8407F2FD0B0F5405F54D0B0F5404F79D03A
S31508002DE8002008BD594BD3F89030034043EA004009
S31508002DF8574B98420FD0B0F1C01F14D0403B9842A9
S31508002E0806D0FFF701FFFFF7B9FEFFF7C3FEE8E7AD
S31508002E18FFF7FAFEE5E74D4B1B6813F0020F40F083
S31508002E2881800020DDE7494B1B6F13F0020F7BD129
S31508002E380020D6E7454BD3F89030034043EA0040D4
S31508002E48444B984210D0B0F1032F14D0A3F58073E1
S31508002E58984206D0FFF7D8FEFFF790FEFFF79AFECE
S31508002E68BFE7FFF7D1FEBCE7384B1B6813F0020F24
S31508002E785DD10020B5E7354B1B6F13F0020F58D10B
S31508002E880020AEE7314BD3F89030034043EA0040C0
S31508002E98314B984210D0B0F1302F14D0A3F5805397
S31508002EA8984206D0FFF7B0FEFFF768FEFFF772FEF6
S31508002EB897E7FFF7A9FE94E7244B1B6813F0020F60
S31508002EC83AD100208DE7214B1B6F13F0020F35D13D
S31508002ED8002086E71D4BD3F89030034043EA0040AC
S31508002EE81E4B984210D0B0F1C02F14D0A3F58043DA
S31508002EF8984206D0FFF788FEFFF740FEFFF74AFE1E
S31508002F086FE7FFF781FE6CE7104B1B6813F0020F9B
S31508002F1817D1002065E70D4B1B6F13F0020F12D16E
S31508002F2800205EE70E485CE74FF4004059E70C4876
S31508002F3857E74FF4004054E7094852E74FF4004072
S31508002F484FE707484DE74FF400404AE70038024084
S31508002F588000C0000002000300200030008000C086
S31508002F680024F40038B5036813F0010F75D10D462F
S31508002F78044603683C4A1A404B68C9680B432969E2
S31508002F880B43A9690B4313430360AB68426822F4F1
S31508002F984052134343606B69826822F440721343B4
S31508002FA88360324B984216D0314B984227D0314B22
S31508002FB8984228D0304B984229D0304B98422AD08C
S31508002FC82F4B98422CD02F4B98422ED02E4B9842F6
S31508002FD830D0012042E00320FFF72CFE00283ED01F
S31508002FE82B68002B3DD0AA69B2F5004F27D000EB15
S31508002FF85300B0FBF3F080B2E06000202EE00C200E
S31508003008FFF718FEEAE73020FFF714FEE6E7C020C8
S31508003018FFF7DAFEE2E74FF44070FFF7D5FEDDE783
S315080030284FF44060FFF706FED8E74FF44050FFF725
S31508003038CBFED3E74FF44040FFF7C6FECEE75A0863
S3150800304802EB4000B0FBF3F04FF6F0730340C0F311
S3150800305842001843E060002000E0012038BD012046
S31508003068FCE70120FAE700BFF369FFEF001001400B
S315080030780044004000480040004C00400050004012
S315080030880014014000780040007C004008B500F0B4
S31508003098C7FB08BD10B5164B08221A7000225A70CD
S315080030A8272199706921D9705B21197145215971B0
S315080030B8104C114921600121616022826361A26175
S315080030C8E2614FF4000323622046FEF7DBF8042387
S315080030D80A4A0B492046FDF718FF0423094A0A49F4
S315080030E82046FDF74BFF2046FEF7F6F910BD00BF50
S315080030F8740000202C06002000800240641F00206F
S315080031089406002014070020E41E0020074A1178B8
S31508003118074B19705178597091789970D178D97088
S315080031281179197152795A71704700BF74000020D5
S31508003138B8050020064B1A7802705A7842709A78B1
S315080031488270DA78C2701A7902715B7943717047AE
S315080031587400002038B51248FDF7D6FF10B10024D0
S31508003168204638BD0E4DAC8F2246296C0D4802F014
S31508003178CCFB2A6B136843F0004313600023AB6348
S315080031882B6841F214029A5812F0800FE8D041F2DF
S3150800319814028021995041F2080200219950DFE76C
S315080031A82C060020C837002038B5194BDC6A00F011
S315080031B837FB00F1FA052368002B07DA00F022FC32
S315080031C800F02EFBA842F6D9012300E0002383B1BC
S315080031D80F4B1B6841F214029A5812F0200F07D0B9
S315080031E841F214022021995041F204020021995013
S315080031F838BD084B1D88064CE36A2A46064998686E
S3150800320802F083FB29462046FDF7EEFEE0E700BFFD
S315080032182C06002034370020C837002072B67047BD
S3150800322862B6704708B5FFF7F9FF08BD10B500F094
S3150800323805FAB8B1FDF79CF9B8B100F099FBFDF7A6
S31508003248ADFC00F0C3FA00F0FDF9094B0340094A42
S31508003258936000F0F7F94468FFF7E2FFA04700F02B
S31508003268C1FB01E000F0BEFB10BD00F0BBFBFBE7AD
S3150800327880FFFF1F00ED00E070B508E04D1C461CF6
S315080032880B78037000F0BEFB304629462246531ECB
S315080032989CB2002AF2D170BD38B50546002401E073
S315080032A80134E4B20A2C15D800F0ACFB04EB44024E
S315080032B89300094AD358AB42F2D804EB440291006A
S315080032C8054A0A4452681344AB42E9D9024B0B44EF
S315080032D8187A00E0FF2038BD6859000808B5C1F318
S315080032E8080353B903688B4209D040F8041B4FF406
S315080032F80072FFF7C1FF012000E0002008BD012089
S31508003308FCE72DE9F0410746FEF794F900247F2CDF
S3150800331814D83E68A30006EB03083B445D6800F032
S3150800332871FB2A46002341460220FEF7D9F938B927
S3150800333856F82430AB4209D10134E8E7012400E005
S315080033480024FEF78FF92046BDE8F0810024F8E747
S3150800335838B50D460C4B984211D004460B4B99428A
S3150800336807D1094C29462046FFF7B8FF48B1204639
S3150800337838BDFFF7C6FF0028F4D10024F7E7044C48
S31508003388F0E70024F3E700BF800200200080000869
S315080033987C0000202DE9F04106460C4617461D46D6
S315080033A8DFF8748001EA08080368B3F1FF3F07D01D
S315080033B8336843450BD13368E41A3444043415E0BA
S315080033C84146FFF78BFF03460028F1D11FE0414627
S315080033D83046FFF7BDFF06460028ECD1002316E065
S315080033E817F8013B04F8013B013D0FD000F00AFB32
S315080033F8331DE31AB3F5007FF2D308F5007130469A
S31508003408FFF7A6FF064628B1041DE9E70123184673
S31508003418BDE8F0810023FAE700FEFFFF70B586B025
S3150800342804460E4600230093884219D80125ECB1B4
S315080034380B2E1FD8DDB10023019302230593012320
S315080034480493FEF7F7F8B4420DD800F0DBFA0394B4
S31508003458694601A8FEF7DCF920B90134E4B2F2E7B7
S315080034680025E4E70025FEF7FDF800E000252846D4
S3150800347806B070BD0025FAE74FF0FF33024A13601D
S31508003488024A1360704700BF7C00002080020020B3
S3150800349870B54B1E144C241AA34201D9002070BDDE
S315080034A816460D460446FFF7F7FEFF2818D02819D2
S315080034B80138FFF7F1FEFF2814D00C4B23400C4ABD
S315080034C8934206D02B46324621460A48FFF762FF42
S315080034D8E5E72B46324621460748FFF75BFFDEE756
S315080034E80020DCE70020DAE7FFFF1F0800FEFFFFE1
S315080034F8008000087C000020800200204A1E0D4B30
S315080035081B1A9A4201D90020704770B50C46054621
S31508003518FFF7C2FE064660190138FFF7BDFEFF2809
S3150800352818BFFF2E01D1002070BD01463046FFF7AF
S3150800353875FFF9E7FFFF1F08104B1B68B3F1FF3F3C
S315080035481AD000B583B00D4A536891680B44D16800
S315080035580B4411690B4451690B4491690B44D269B0
S3150800356813445B4202AA42F8043D04210448FFF7C3
S315080035788FFF03B05DF804FB012070478002002026
S31508003588F88100080D4B1B680D4A12681A440D4B42
S315080035981B6813440C4A126813440C4A12681A44E6
S315080035A80B4B1B681A440B4B1B6813440A4A1268D0
S315080035B8DA4201D0002070470120704700800008D1
S315080035C804800008088000080C800008108000089D
S315080035D81480000818800008F881000808B50D4B03
S315080035E81B68B3F1FF3F0BD10B4B1B68B3F1FF3FC9
S315080035F80DD00948FFF785FE034648B1012307E0C1
S315080036080448FFF77EFE03460028EDD100E00123B3
S31508003618184608BD800200207C0000200048704734
S315080036280080000808B5FFF727FF08BD08B5FFF7AB
S315080036382FFF08BD08B5FFF761FF08BD08B5FFF7F6
S31508003648A1FF08BD08B5FFF7E9FF08BD08B5FFF7EC
S3150800365873FF034608B9184608BDFFF7BFFF0346B8
S31508003668F9E70000054BDB6913F0200F04D0034B7C
S315080036785B6A0370012070470020704700480040C5
S3150800368810B5094B986200F0CBF800F10A04064B0E
S31508003698DB6913F0800F05D100F0B4F900F0C0F823
S315080036A8A042F4D910BD00BF0048004010B588B044
S315080036B80C4C236823F0010323604FF461430193FC
S315080036C800230293039304930C2205920693079307
S315080036D801A92046FFF746FC236843F00103236047
S315080036E808B010BD0048004070B506460D4640298A
S315080036F804D82846FFF7C4FF00240BE083210748AF
S3150800370800F09AF8F5E700F07DF9305DFFF7B8FFA5
S315080037180134A4B2ABB2A342F5D870BDEC5900087F
S3150800372870B5254B1C78BCB92448FFF79BFF0128C0
S3150800373801D0204670BD214B1B78013BDBB23F2BDD
S31508003748F7D800F06DF81E4B18601E4B00221A7049
S31508003758194B01221A70ECE706460D46194B1B78D9
S31508003768013316481844FFF77DFF0446012815D18A
S31508003778144B1A780132D2B21A70104B1B789A4237
S3150800378801D00024D5E710493046FFF775FD0A4BE6
S3150800379800221A700B4B1B782B70CAE700F040F80A
S315080037A8074B1B686433984203D90024024B1C70E4
S315080037B8BFE70024BDE700BFC50400208404002035
S315080037C8C8040020C604002085040020024B0022F5
S315080037D81A605A609A60704710E000E008B5FFF76B
S315080037E8F5FF054B054A5A6000229A6005211960BB
S315080037F8034B1A6008BD00BF10E000E0BF4B03008A
S31508003808CC040020044B1B6813F4803F03D0034AFA
S31508003818136801331360704710E000E0CC040020F9
S3150800382808B5FFF7EFFF014B186808BDCC04002060
S3150800383808B5FFF7F5FF08BD08B500F0E3F8FCE79B
S3150800384808B500F0C7F8012803D00B4B1B78012BE5
S3150800385800D008BDFFF7E4FF084B1B68084A126842
S31508003868134403F5FA739842F3D3034B00221A70EC
S31508003878FFF7DCFCEDE700BFD4040020D0040020E5
S31508003888D8040020014B1860704700BFD0040020F8
S31508003898014B1868704700BFD004002008B5054BCF
S315080038A81B78012B00D008BDFFF7BAFF024B18603A
S315080038B8F9E700BFD4040020D804002008B5044B53
S315080038C801221A70FFF7EAFFFFF7BAFF08BD00BF23
S315080038D8D404002008B5FFF7A5FC00F08FF8FFF719
S315080038E87DFFFFF79FFE00F00DF8FFF7E7FF08BD1D
S315080038F808B500F087F8FFF785FF00F00FF8FFF71F
S315080039089FFF08BD08B500F07BFBFFF7CFFE024B0B
S3150800391800221A7008BD00BF4C00002000B583B00D
S315080039280DF107011048FFF7FBFE012809D00DF134
S3150800393807010D4800F092F901280BD003B05DF88D
S3150800394804FB0A4B00221A709DF80710064800F077
S3150800395877FBECE7054B03221A709DF80710024817
S3150800396800F06EFBEAE700BFDC0400204C000020EC
S315080039787047000038B504460D46094B1B7833B125
S31508003988074B1B78032B06D000F052FB38BDC9B28B
S31508003998FFF7AAFEF4E7E9B2204600F03BF9F3E799
S315080039A84C000020044B1B78013B012B01D9402011
S315080039B870470020704700BF4C000020044B1B7856
S315080039C8013B012B01D9402070470020704700BFF2
S315080039D84C00002008B500F021FB034600B101237E
S315080039E8184608BD08B500F005F9034B03221A70F6
S315080039F8FFF754FF08BD00BF4C00002008B5FCF7C8
S31508003A08C9FD08BD08B5FCF7CAFD08BD10B5FFF71E
S31508003A18A1FBB8B9FFF704FF464B1B68984209D3C0
S31508003A2803F5FA73434A13600024002C37D00024A0
S31508003A38002C4AD0FFF7F4FE3F4B1B68984259D230
S31508003A48002460E03D4A10803D4B9C894FF4006095
S31508003A5800F0A8FE844213D0394B9C8940F606002C
S31508003A6800F0A0FE8442D5D101F0EEFD334B1B8849
S31508003A78002BCFD0FFF798FB304B00221A80C9E7F6
S31508003A88012000F0C9FE2D4B1B88002BC2D001F07F
S31508003A984BFEFFF789FB294B00221A80BAE76823F1
S31508003AA8284A03FB0423284A1360022000F0B4FEC0
S31508003AB8224B1B880BB90134B7E701F035FEFFF72F
S31508003AC873FB1E4B00221A80F5E7204B03EB841381
S31508003AD81F4A1360052000F09FFE184B1B880BB978
S31508003AE80134A5E701F020FEFFF75EFB134B002221
S31508003AF81A80F5E742F210721A440F4B1A6001F061
S31508003B086FFD9DE70134A4B968230E4A03FB042315
S31508003B180D4A1360032000F07FFE084B1B88002B14
S31508003B28F0D001F001FEFFF73FFB044B00221A8094
S31508003B38E8E710BD280500201C05002034370020BA
S31508003B48C8370020503700204C3700200C3E00208C
S31508003B58443700201F4B1B7803B1704710B5FFF791
S31508003B6899FAFFF75DFE00F5FA701B4B1860FFF728
S31508003B7857FE42F210730344184A136000F0BAFD60
S31508003B88174A002313805380164A13805380164A0F
S31508003B98138053804EF6030000F0ECFDFFF7B6FAE3
S31508003BA8124C2046FFF7C6FA0621204600F0DAFB33
S31508003BB800F0F6FBFFF76CFE42F20F73984203D942
S31508003BC80B4B01221A7010BD42F21070FFF75AFE0D
S31508003BD8F6E700BF4D000020280500201C05002038
S31508003BE8C4370020C0370020BC3700202005002035
S31508003BF82605002008B5054B00221A70044B1B78C9
S31508003C0803B108BDFFF7A6FFFBE700BF4D0000207C
S31508003C18260500200F4B1B78012B00D0704770B47F
S31508003C280D4B1C68E6692662002306E01A1DC55C6A
S31508003C38224482F8205001339BB28AB29A42F5D8B8
S31508003C480432A4F86420012384F866301E44E66129
S31508003C5870BC7047260500204C37002008B5044B71
S31508003C681B78012B01D0002008BDFFF7CFFEFAE725
S31508003C782605002010B5294B1C68294B1B7813F01C
S31508003C88400F2AD113F0010F02D0002284F86720CA
S31508003C9813F0040F03D094F86730012B27D0204B74
S31508003CA81B7813F0080F03D094F86630012B25D03B
S31508003CB81B4B1B7813F0020F18D01A4B19880B1FC9
S31508003CC8402B13DC94F8673083B9174B1868043906
S31508003CD8C9B2043000F0B4F908E00123E36100230F
S31508003CE8A4F8643084F8663084F8673010BDB4F8F0
S31508003CF8641004F1200001F0DFFBD0E7002384F804
S31508003D086630B4F864100029D2D0012384F86730E5
S31508003D1804F1200001F0D0FBCAE700BF4C370020A9
S31508003D28403700203437002048370020014B00224E
S31508003D385A7070472C050020034BFE22DA7018715A
S31508003D480222A3F8442070472C05002010B5054C1C
S31508003D5800232370FFF7EAFFFF23E3700123A4F883
S31508003D68443010BD2C050020064BFF22DA700022CD
S31508003D781A71597859719A71DA711A720622A3F862
S31508003D88442070472C05002008B50020FFF7D4FF0B
S31508003D9808BD0000074BFF22DA70074A9A6400221A
S31508003DA81A715A719A710722C3F807200822A3F8CC
S31508003DB8442070472C0500202C5A0008044BFF2283
S31508003DC8DA7042689A640122A3F84420704700BF53
S31508003DD82C05002008B53120FFF7AEFF08BD000006
S31508003DE838B5084CFF23E370002525716571FFF780
S31508003DF8D9FDA071E571257265720723A4F84430C8
S31508003E0838BD00BF2C05002038B5FFF78FFF0E4CCC
S31508003E1801252570FF23E37010232371002363719E
S31508003E28FFF7C0FDA071FFF7C9FDE071FFF7C6FDF2
S31508003E38C0F3072020726572A5720823A4F84430D7
S31508003E48FFF7F0FB38BD00BF2C05002038B505463E
S31508003E584478FFF7A7FD0138844210DC0A4C6A78D3
S31508003E68A16C201DFFF708FAFF23E3706A78A36C94
S31508003E781344A3646B780133A4F8443038BD222070
S31508003E88FFF75AFFFAE700BF2C05002038B50446A5
S31508003E984578FFF787FD0138854211DC61680A4DC8
S31508003EA8A9646278281DFFF7E7F9FF23EB706278A3
S31508003EB8AB6C1344AB6463780133A5F8443038BD5A
S31508003EC82220FFF739FFFAE72C050020F8B5054642
S31508003ED81746002406E015F8013B1C44E4B2FFF730
S31508003EE891FD31464E1E0029F5D13C600120F8BDEA
S31508003EF810B5084CFF23E370E21D4168A06CFFF774
S31508003F08E5FF207100236371A3710823A4F84430E0
S31508003F1810BD00BF2C05002038B505460D4B9C6C16
S31508003F28FFF740FD6A1C411E2046FFF77FFB60B17C
S31508003F38084CFF23E370FFF735FD0138A36C0344EB
S31508003F48A3640123A4F8443038BD3120FFF7F4FEF2
S31508003F58FAE700BF2C05002038B504464578FFF770
S31508003F6821FD023885420EDC114BFF22DA70012248
S31508003F78A3F84420617851B9FFF768FB30B93120B6
S31508003F88FFF7DAFE02E02220FFF7D6FE38BDA21CAC
S31508003F98074B986CFFF74AFB28B16178044A936C7B
S31508003FA80B449364F2E73120FFF7C6FEEEE700BF3D
S31508003FB82C05002008B54168074B986CFFF73AFBB3
S31508003FC830B1054BFF22DA700122A3F8442008BD58
S31508003FD83120FFF7B1FEFAE72C05002008B5FFF7F0
S31508003FE825F9034BFF22DA700122A3F8442008BDFD
S31508003FF82C05002008B589B2FFF7BCFC08BD0000EF
S31508004008054B00221A709A6483F84320A3F84420C3
S315080040189A705A70704700BF2C050020034B1B780E
S315080040280BB1012070470020704700BF2C050020FF
S31508004038024B002283F84320704700BF2C05002056
S3150800404808B50378FF2B04D0354A1278012A14D00C
S3150800405808BDFFF7D9FE324B93F84330012B5AD0E7
S315080040682F4BB3F944100029F2DD1846012380F8CE
S3150800407843300330FFF7BEFFEAE7C93B352B46D87E
S31508004088DFE803F03345454245453F363C39454563
S3150800409845454545454545454545454545454545BA
S315080040A84545454545454545454545454545241EF2
S315080040B81B2145454527452A2D30FFF7C7FECAE780
S315080040C8FFF7E4FEC7E7FFF779FEC4E7FFF710FF37
S315080040D8C1E7FFF75FFEBEE7FFF756FEBBE7FFF748
S315080040E843FEB8E7FFF732FEB5E7FFF715FFB2E775
S315080040F8FFF732FFAFE7FFF773FEACE7FFF75AFFA4
S31508004108A9E7FFF76BFFA6E7FFF764FEA3E72020FA
S31508004118FFF712FE9FE71020FFF70EFEA0E700BF85
S315080041282C05002035230370012343708170033062
S31508004138704700003623037004234370024BDB697B
S31508004148C0F802300630704778050020322303701D
S3150800415804234370024B5B6AC0F802300630704786
S3150800416878050020372303700323437001228270E1
S31508004178C3700623037105307047FF2303700130A7
S31508004188704700000346014400208B4234D210B41D
S3150800419810E0362A23D0FF2A2BD0352A05D198785D
S315080041A803E0D3F80240154A94625A780232134457
S315080041B88B421ED21A78332A16D0EAD8032A04D094
S315080041C8062A07D0012AF0D1EBE7D3F802400B4AB2
S315080041D81463EAE7D3F80240084AD462E5E7D3F855
S315080041E80240064AD461E0E7D3F80240034A14625B
S315080041F8DBE75DF8044B7047704700BF7805002079
S31508004208074B828C1A80C28C5A80064B028D1A80FC
S31508004218428D5A80044B028E1A80428E5A80704705
S31508004228C4370020C0370020BC370020F8B504463C
S31508004238012303704370184B9A6982700025C5706C
S31508004248164A12684260058180274781144A12680F
S31508004258C2600561456185619E69324659691C30A7
S3150800426801F053FB06F118002044C6F1100229464E
S31508004278043001F055FB4022294604F12C0001F0D0
S315080042884FFB3A46294604F16C0001F049FB054BF9
S315080042981B68C4F8EC30F8BD78050020385A0008C1
S315080042A8C4370020345A000838B50A4C2568284609
S315080042B8FFF7BCFF012105F1F000FFF733FFFFF711
S315080042C851FFFFF75AFF2368C11A184601F0F4F898
S315080042D838BD00BF4837002038B50B4C2568284636
S315080042E8FFF7A4FF032105F1F000FFF71BFFFFF70F
S315080042F821FFFFF72BFFFFF740FF2368C11A18466F
S3150800430801F0DAF838BD00BF4837002010B5114B60
S315080043181C682378022B01D0002010BD04220E4900
S31508004328A01801F0E3FA98B90C4B9A69596904F18F
S315080043381C0001F0DBFA08B10020EEE72269074BFA
S315080043485A62074B198804F1F000FFF71BFFE4E7E8
S315080043580020E2E748370020385A00087805002088
S315080043683437002010B582B00C4C6061A161002377
S31508004378A3704FF6FF73ADF80430ADF806304FF466
S31508004388864101A801F048F8606010B14FF48843E7
S315080043988380024B00221A8002B010BD78050020DF
S315080043A8024B00221A805A80704700BFC437002083
S315080043B838B5984B1B88B3F5937F15D059D840F272
S315080043C80F12934200F09A80B3F5887F47D3B3F566
S315080043D8887F00F0978040F22512934240F01581B5
S315080043E88C4B4FF493721A808B4B1B7813F0020F81
S315080043F800F0CB80884B1B7813F0020F40F0CD8075
S31508004408844B1B6942F21072934200F3CF80814AAB
S3150800441803F57A7313619378032B40F0A9807D48D6
S31508004428FFF7EEFE7B4D288C00F0BCF90404688C77
S3150800443800F0B8F9204340084FF47A7404FB00F0FA
S315080044480028C0F2B7802861724C216904F1080077
S3150800445801F014FA40F255132380032075E0002B67
S3150800446840F0D3806B4B01229A704FF47A721A6126
S315080044785FE0B3F5AB7F3AD030D9B3F5B57F00F036
S31508004488A78040F26B12934240F0BF80624B1B78BC
S3150800449813F0020F00F0A1805F4B1B7813F0020F90
S315080044A840F0A3805B4B1B6942F21072934200F3FB
S315080044B8A880584A03F57A7313619378032B00F09A
S315080044C89C80FFF709FF534C216904F1080001F0A5
S315080044D8D5F94FF4B5732380032036E040F2551218
S315080044E8934240F092804B4B4FF4AB721A804B487C
S315080044F801F0CBF9002862D1002026E0454B4FF49D
S3150800450888721A80444B1B7813F0020F1ED0424B50
S315080045181B7813F0020F20D13E4B1B694EF65F221B
S31508004528934202DC5B003B4A13613A4B9B78022BA9
S315080045381AD0FFF7B9FE374C216904F1080001F0D3
S315080045489DF940F20F132380032038BD334801F044
S315080045589CF90028DBD10020F7E7FFF7D7FE0228E9
S31508004568DAD12C4B02229A702A4B4FF47A721A61C6
S31508004578FFF7B2FE274C216904F1080001F07EF91D
S3150800458840F2251323800320DFE7244801F07DF94C
S3150800459800287FF42FAF0020D7E7FFF7B7FE0528D6
S315080045A87FF42EAF1B4B03229A7038E70020194B6D
S315080045B81880CAE7174B6FF000421A6144E7154B93
S315080045C802229A704FF47A721A61FFF7E9FE78E7C1
S315080045D8104B40F26B121A8058E7104801F055F94B
S315080045E800287FF459AF0020AFE7FFF78FFE0528AC
S315080045F87FF458AF074B03229A700648FFF700FE68
S3150800460810E70020034B18809FE7024B00221A8008
S3150800461802209AE778050020403700208005002008
S3150800462808B5FFF7C5FE08BD10B4013A0A4400E00C
S31508004638023191420BD20C784B7803EB04239BB2D8
S31508004648184480B28342F3D9013080B2F0E702D029
S315080046585DF8044B70470B781B02184480B28342F6
S31508004668F6D9013080B2F3E770B4C5780D44EDB2D7
S31508004678134CE57083780E0A3344DBB2A37042788C
S315080046886270007820709CB2A64206D90132D2B26E
S315080046980B4C62700AB901302070C9B28D420CDA27
S315080046A80133DBB2064A93703BB953780133DBB260
S315080046B8537013B913780133137070BC704700BF71
S315080046C83C37002010B5094C2368014603F1080059
S315080046D8FFF7CAFF2368064A117819725178597282
S315080046E891789972D278DA7210BD00BF4C370020DB
S315080046F83C3700201A4B00221A7006E0194A002196
S3150800470822F813100133164A1370154B1B78002B21
S31508004718F4D0134B00221A7008E01349682202FBEA
S3150800472803120021517601330D4A13700C4B1B787E
S31508004738002BF2D00D4B4FF480621A80084B0022EA
S315080047481A7007E00A4A02EB8312002191800133A6
S31508004758034A1370024B1B78002BF3D0704700BF2F
S31508004768AC050020B837002050370020B4050020D3
S315080047780C3E0020094B00221A70084B1B7863B9B7
S315080047881946074A32F813201AB10133034A137037
S31508004798F3E7034B23F8110070477047AC05002070
S315080047A8B8370020030A43EA002080B270470000A1
S315080047B808B5142205490020FFF736FF10B1FFF7A0
S315080047C8F1FF08BD4FF6FF70FBE700BFD63700209C
S315080047D838B50D4D2B7C6C7C04EB0324A4B2143C31
S315080047E8A4B22044082205F11A0180B2FFF71CFF7B
S315080047F8224605F12201FFF717FF10B1FFF7D2FF8E
S3150800480838BD4FF6FF70FBE7C837002008B5062005
S31508004818FFF7DEFF08BD000070B5B24B1C68042818
S3150800482800F09681B04BB14A1360B14A1360032869
S3150800483859D0022800F0C880052800F07281AD4BCF
S315080048489B7B452B54D1AB4A157C537C03EB05213E
S31508004858A94A128891424BDC8DB2A74B1D80A54BFD
S315080048681B7D13F03F0F43D1A24B5B7D002B3FD135
S31508004878A24B1C880CB95B884BB19E4BDB8B9C42C0
S3150800488836D19C4B1A8C9D4B5B889A4230D1FFF7E0
S315080048988FFF4FF6FF7398422AD1964BDB7D062B7E
S315080048A800F0E981112B00F09F81012B20D1914B53
S315080048B893F82230082B1BD18E4B002283F822202E
S315080048C89B8C4FF6F672934240F28A810933894ADD
S315080048D89384884B5A8BDA839A8B1A845C83874A23
S315080048E852889A8378E1637E03F00F03032B05D079
S315080048F80023814A1380824A137070BD238A002BCD
S31508004908F6D17F4B08221A70FFF7B4F97C4B1B784F
S3150800491813F0200F00F0A48400237A4A13806376E4
S31508004928744B142283F82F20734B28221A80714B54
S31508004938502283F82E20227A6E4B83F82A20627A30
S3150800494883F82B20A27A83F82C20E27A83F82D2084
S31508004958227B83F82620627B83F82720A27B83F8AC
S315080049682820E27B83F829200622DA75A2885A8449
S31508004978E2889A84614A1188598352889A832288D8
S31508004988DA8362881A84637E13F0100F00F0348580
S31508004998584B002283F8312083F83020554C4023A1
S315080049A8A375554B1B881A0A22746374002384F866
S315080049B8353084F8343084F8323084F83330FFF7E9
S315080049C825FFC0436086F2E04F4AD3780133DBB24D
S315080049D8D37063B993780133DBB293703BB95378D4
S315080049E80133DBB2537013B91378013313700023FC
S315080049F8414A1380434A1380637E052B18BF072B49
S31508004A0809D1A37E0133DBB2A376782B7FF470AF86
S31508004A18002363766CE7002B3FF46AAF228A002AE4
S31508004A2874D0A27E511EA176002A7FF461AFE27E79
S31508004A38082A27D0591EC9B2012921D91046042A9D
S31508004A4828BF042003218140A1760132E27603F0CB
S31508004A580F03013B072B3FF64BAF01A252F823F091
S31508004A68294F0008A54A0008E14A0008DD51000850
S31508004A78F9480008DD510008F9480008DD51000822
S31508004A88052ADBD1002363761D4B80221A70FFF7AF
S31508004A98F1F8184B142283F82F2045E7154B002206
S31508004AA883F82F20134B93F82F2042F0020283F83D
S31508004AB82F20022283F83620042283F8372006227C
S31508004AC883F838200A2283F839200B4A2C211180CA
S31508004AD8602283F82E202EE7094B04221A70FFF766
S31508004AE8C9F8E2E34C370020FE3700204837002093
S31508004AF838370020C837002034370020C43700204C
S31508004B08403700200A3E0020B005002003F00F03B6
S31508004B18032B7FF4EDAEAC4B08221A70FFF7AAF800
S31508004B28F4E6AA4B1B689B88002B3FF4E1AE0023EA
S31508004B38A74A1360A74AA8490A60A8490A60A84A62
S31508004B481380A84A1380A04B08221A70FFF768FD3D
S31508004B58A34B1A88002A3FF4CBAE02F11C0189B28E
S31508004B68A04B1980A04B080A187459749749096804
S31508004B78087A98751120D875083292B2100A40EA50
S31508004B880222DA84002283F8282083F829208A88D2
S31508004B985A84CA889A84954A1088588352889A8368
S31508004BA80A88DA834A881A8436338B4A13608E4C05
S31508004BB84523A3730022E273627522758C490B8814
S31508004BC801339BB20B80190AA174E37422766276C4
S31508004BD8FFF7EEFDC04320837B4B00221A708CE654
S31508004BE80833814A938474E61C3D7E4B1D80774BB7
S31508004BF8804A1A600EE01A880AB9598829B34FF606
S31508004C08FF718A421ED07849498B8A422DD0403393
S31508004C186E4A13606D4B1B68774A9342BFF468AEB9
S31508004C289A88002AF3D07049898C8A42EFD1DA88A3
S31508004C38002AE0D06C49498C8A42DCD0B2F58A4F02
S31508004C48E5D1D8E758888842DDD10023604A136041
S31508004C585D4A022111705F4A5F490A605F490A6026
S31508004C685F4A1380FFF7DCFC72E75F4A918B5A8824
S31508004C789142CCD1E9E7FFF7C9FD4FF6FF73984291
S31508004C887FF436AE5D4C5D4B9C425AD9564B93F829
S31508004C982F3003F03F03022B7FD0534B93F82F3066
S31508004CA813F0040F7FF424AE4F49142381F82F30EC
S31508004CB84C4B28221A80502381F82E3091F8290067
S31508004CC891F82D3081F8293091F8282091F82C3060
S31508004CD881F8283081F82C2091F8273091F82B4054
S31508004CE881F8274081F82B3091F82640444D2C70DE
S31508004CF891F82A5081F8265081F82A400130C0B226
S31508004D0881F82D0060B90132D2B281F82C203AB95F
S31508004D180133DBB281F82B3013B9013481F82A4004
S31508004D28314B5A8C37490A80998C59849A845A8BFC
S31508004D38DA839A8B1A842D4A1188598352889A835A
S31508004D482CE6617E21B1284B9A8CA3889A4201D019
S31508004D58683498E7244B5A8CE3889A42F8D1224B50
S31508004D685A8B23889A42F3D11F4B9A8B63889A42A7
S31508004D78EED1174B1C60144B00221A701A4B93F885
S31508004D882F2012F0040F00F0DA80002363760E4B0A
S31508004D9820221A70FEF76EFFAAE5134B9B8C99B270
S31508004DA8184A1380164B00221A70154B1B78002BCD
S31508004DB87FF473AF144A32F81320914226D0013390
S31508004DC80F4A1370F1E700BF403700204437002028
S31508004DD84C370020F23700204837002038370020A3
S31508004DE80A3E002034370020C8370020C437002080
S31508004DF8AE0500200C3E00204C3E0020503700200F
S31508004E08AC050020B6050020B837002000249A4BC8
S31508004E181C700BE019469948682202FB0302527E69
S31508004E284AB1072A56D00133934A1370924B1B7816
S31508004E38002BEFD002E0682404FB0104002C3FF4A1
S31508004E4857AD8F4B1C600323A37623760023A375DF
S31508004E580422E275E3768B4DAB8CA3806B8CE380DA
S31508004E686B8B2380AB8B638001206076864B1A7820
S31508004E7822735A7862739A78A273DB78E37320826E
S31508004E8895F82930E37295F82830A37295F82730F3
S31508004E98637295F826302372FFF714FC95F82E00EE
S31508004EA800F0F003502B3BD9734B00221A70724B53
S31508004EB81B781A4601090539B3EB810F30DA03F175
S31508004EC83601704D695C59B3012911D101336A4A13
S31508004ED81370ECE73CB16949682202FB0312917E1C
S31508004EE8A27E91429FD96824644A04FB03249AE760
S31508004EF802291AD103F13701624D695C042914D1D4
S31508004F0802F13801695C3932AB5C43EA01235F4A2E
S31508004F18138040F20A62934228BF13466382A3822B
S31508004F28584B102283F82F20BCE503F13702554960
S31508004F388A5C002AF4D013444F4A1370B7E7514BDA
S31508004F4893F82E301B099B004B480370EB1A9BB24B
S31508004F58143B9BB24E48038001F00F01022903D186
S31508004F6802F03F0112290FD013B912F0030F0BD024
S31508004F78444BD98C2389994240F0E781414B198DD6
S31508004F886389994240F0E18112F0100F47D0218ACF
S31508004F98002944D004F10C00FFF766FB394B93F857
S31508004FA82A303C4A1078834239D1364B93F82B304D
S31508004FB851788B4233D1334B93F82C3092789342FD
S31508004FC82DD1304B93F82D50324BDB789D4226D1A4
S31508004FD820736173A273E373E37ECBB9237EA27E43
S31508004FE89B1ADBB2A17DA3EBD103DBB25AB21944F3
S31508004FF8C9B2A175002A01DA5B425AB2E07DA2EB72
S31508005008900350FA83F3DBB2E37503EBD1032376F7
S31508005018214B01221A70237EA37600232382617E00
S3150800502801F00F03013B072B3FF662ACDFE813F0EC
S3150800503808003800AC007001BA01D8018D01610179
S31508005048154B1B7813F0010F3FF452AC0323637614
S31508005058114B40221A70002323820D4B188820B161
S315080050680D4B42221A70FFF72DFB0C4B00221A80B3
S31508005078FEF700FE4AE400BFAC05002050370020C2
S315080050884C370020C8370020B0050020B605002098
S31508005098343700203C370020403700200A3E0020DD
S315080050A8AD4B1B7813F0010F64D0AC4B93F82F3037
S315080050B803F03F03122B5DD1A84B93F82E0000F09E
S315080050C8F003502B2DD9A64B00221A70A44B1B7837
S315080050D81A4601090539B3EB810F22DA03F13601BD
S315080050E89E4D695CE9B1012903D101339C4A1370C5
S315080050F8ECE7022934D103F13701984D695C042994
S315080051082ED102F13801695C3932AB5C43EA0123D6
S31508005118944A138040F20A62934228BF1346638270
S31508005128A382032363768D4B93F82620227293F87D
S315080051382720627293F82820A27293F82930E3721E
S315080051480120FFF7BFFA844B42221A7000232382F4
S31508005158854A1380854A1380FEF78CFDFFF7D6BB70
S3150800516803F137027D498A5C002ADAD013447C4A5F
S315080051781370ABE7784B20221A70FEF77BFD7C4B41
S315080051881B6800225A7688E5744B93F82F3013F07B
S31508005198010F25D011F0100F22D1238A002B7FF496
S315080051A8A7AB714D2888013080B2FFF78BFA6A4A97
S315080051B8137843F0100313702A881AB143F00203D0
S315080051C8654A1370FEF756FD012323820823637682
S315080051D80023E376614B112283F82F20FFF7A4BB3F
S315080051E813F0200F0FD05D4890F834301A0290F863
S315080051F8353042EA03065F4D2868304428605A4825
S315080052080288931B0380584B188848B111F0100F71
S3150800521806D1514A137843F002031370FFF752FA7E
S315080052284E4B93F8302093F8313003EB02239BB2A8
S315080052384C4A1380A28A934200D80BB9494B1A8064
S31508005248484B1B886382444B1B7813F0030F3FF4C3
S315080052584FAB464B00221A80FEF70CFDFFF756BBEC
S3150800526813F0100F0DD00023404A13800122228222
S3150800527804226276E376394B112283F82F20FFF74A
S3150800528853BB3A4A128872B113F0010F01D00023B2
S315080052982382238ADBB9638A9A4201D9334A13805F
S315080052A8324B1B8823820023E376334B1A68314B2B
S315080052B81A602E4B1B886BB1238A5BB128332A4A9E
S315080052C81380264B182283F82F20FFF730BB274A6E
S315080052D81380E8E7204B1B7813F0020F3FF408AB5E
S315080052E8214B28221A801D4B102283F82F20FFF7FE
S315080052F81EBB194B1B7813F0010F3FF4F9AA0023BC
S315080053086376154B10221A70FEF7B4FCFFF7F0BA4D
S31508005318154B188808B1FFF7D5F9104B93F82F30B5
S3150800532813F0010F2DD00C4B1B7813F0010F25D065
S31508005338072363760023A37623820120FFF7C2F9A1
S31508005348054B10221A70FEF795FC044B102283F8B9
S315080053582F20FFF7E9BA00BF40370020C8370020DA
S31508005368AC050020B6050020343700200A3E002088
S315080053784C37002048370020383700200623637644
S31508005388DBE7224B1B7813F0010F05D0052363765C
S3150800539800232382FFF7ACBA1D4B1B88002BD4D1F8
S315080053A8FFF7A6BA1A4B188808B1FFF78BF9194BF5
S315080053B893F82F3013F0010F0CD0072363760023D8
S315080053C8A3760120FFF77EF9104B10221A70FEF714
S315080053D851FCBAE70E4B1B88002BB6D1FFF788BAE3
S315080053E80A4B1B7813F0010F3FF482AA072363764A
S315080053F80023A376FFF77CBA064B062283F83020EB
S315080054080A2283F83120FFF7C9BA00BF40370020BF
S3150800541834370020C8370020F8B505460E46234A13
S31508005428138801339BB21380B3F5FA4F03D3134697
S315080054384FF480521A801E4B00221A701C4B1C7897
S315080054486CB91C4B03EB84139F88184B1888FFF715
S31508005458A9F98742E3D00134154B1C70EEE7002200
S315080054681A70134B1B7863B9124A02EB8312928897
S315080054781AB101330E4A1370F3E70E4800EB83108E
S3150800548800E0002068B1094B1A88130A43EA022388
S315080054988380C68035B12B8803806B884380402378
S315080054A80372F8BD00230360F9E700BFB4050020BE
S315080054B8AC0500200C3E002000290CDD08B58AB290
S315080054C8054B1A80054B1B68834203D001461846CC
S315080054D800F01BFA08BD70470A3E0020383700203E
S315080054E8F0B43A4B00221A70394E02E00133374AB3
S315080054F81370364B1B78072B18D8354D5A001A44A3
S3150800550894002E192A5B002AF0D07488002CEDD056
S315080055180588AA42EAD142889442E7D10C687460A1
S31508005528898831812B4B1B78B37222E0274B0022DE
S315080055381A7002E00133254A1370244B1B78072B8F
S315080055480AD8234D5A001A4494002E192A5B002AB1
S31508005558F0D17288002AEDD1082B0CD002683346A0
S3150800556843F8042B0A6872608A889A80194B1B7854
S31508005578B372F0BC70470023174A1370174A1370A2
S31508005588124A137002E00133104A13700F4B1B7846
S31508005598072B11D80F4A147803EB430295000C4AD7
S315080055A82A44927AA61A0C4D2D78AE42EBDD0A4AA1
S315080055B816700A4A1370E6E7084B1B78034A1370F5
S315080055C803EB43039A00024E1644C7E72206002057
S315080055D8C0050020200600202806002021060020F5
S315080055E810B4164B1C780134E4B21C70144B002214
S315080055F81A7002E00133124A1370114B1B78072BF5
S3150800560818D810485A001A4491004218415A528824
S315080056180A43EFD003EB4302910002460A44927A02
S31508005628A21A772AE6DD03EB43018A000146002021
S315080056388850DFE75DF8044B704700BF2006002056
S3150800564822060020C0050020324B1B88292B0CD9BE
S3150800565810B5304B00221A802F4B9B8AB3F5807FF2
S3150800566807D0B3F5007F43D010BD2A4B00221A8015
S315080056787047294BDA8C294B1B889A42F4D1264B5A
S315080056881A8D264B5B889A42EED1254C2146A01DD9
S31508005698FFF726FF002204F8022C022204F8012C40
S315080056A82168C4F80A10A188E1811E4908682060A3
S315080056B88988A18044F8100C24F80C1CD4F80A1020
S315080056C844F8161CE28924F8122CE28822822289D8
S315080056D86282124A1188E18052882281082204F8D7
S315080056E80A2C062204F8092C0A4B2A221A80BBE738
S315080056F8094BDA8C094B1B889A42B5D1064B1A8D89
S31508005708064B5B889A42AFD1054801460630FFF733
S31508005718E7FEA9E734370020C8370020C437002039
S31508005728DE370020B805002030B4494BDA8B4FF62F
S31508005738FF739A421AD0474B1B8847490988534032
S31508005748194208D1424B198C424B5B88424840881B
S315080057584B40184217D0414B414A11881980528844
S315080057685A80404B00221A703F4D13E0384B198C6B
S315080057784FF6FF739942DED1354B3C4A10681860DC
S3150800578892889A8021E0354B1A805980E9E70133D7
S31508005798344A1370334B1B78072B0ED832485A00F5
S315080057A81A44910045182D4A1488425A9442EED153
S315080057B82A4A50886A889042E9D1082B16D0244B81
S315080057C855F8042F1A60AA889A80214B284A116826
S315080057D8C3F8061092885A8108221A7300225A7347
S315080057E8244A13880E33138030BC7047184B4FF081
S315080057F8FF321A609A8000221A629A841C4908683D
S31508005808C3F8060089885981C3F8160059831349CD
S315080058180888D884498819850E4908889883498844
S31508005828D9831A75012159759A73D9730821197478
S315080058385A7406229A740422DA74197306225A7359
S3150800584836330D4A13600B4B2A221A80CCE700BF61
S31508005858C8370020C4370020C03700202406002097
S31508005868BC37002022060020C00500203C5A000844
S31508005878B8050020343700204837002010B50446FC
S315080058884160FDF703FC206010BD10B50446FDF71E
S31508005898FDFB2368C01A63689842B4BF002001203C
S315080058A810BD000070B50D4E0D4CA41BA4100025A4
S315080058B8A54209D10B4E0C4C00F03AF8A41BA410CB
S315080058C80025A54205D170BD56F8253098470135FB
S315080058D8EEE756F8253098470135F2E74C5A00089E
S315080058E84C5A00084C5A0008505A000830B500248B
S315080058F8A24201D1002007E0035D01340D1915F80D
S31508005908015CAB42F4D0581B30BD10B5431E0A449F
S31508005918914200D110BD11F8014B03F8014FF7E782
S3150800592802440346934200D1704703F8011BF9E77E
S31508005938F8B500BFF8BC08BC9E467047F8B500BF66
S30D08005948F8BC08BC9E46704736
S315080059500000000000000000010203040607080911
S315080059600000000001020304008000080080000017
S31508005970010000000000010800800000020000008D
S3150800598000800108008000000300000000000208F3
S3150800599000000200040000000000040800000400E3
S315080059A005000000000008080000040006000000CA
S315080059B000000C08000004000700000000001008A2
S315080059C0000004000800000000001408000004009D
S315080059D00900000000001808000004000A00000082
S315080059E000001C08000004000B000000433A2F5773
S315080059F06F726B2F736F6674776172652F4F706560
S31508005A006E424C542F5461726765742F536F7572CA
S31508005A1063652F41524D434D375F53544D333246DC
S31508005A20372F72733233322E630000004F70656E63
S31508005A30424C540063825363ADDE1223FFFFFFFF1F
S30908005A40FFFF000056
S30D08005A4424A8FF7F0100000001
S30908005A4C1D02000821
S30908005A50F901000842
S31508005A540024F40001000000100000000401000006
S70508000B5196
